:020000040000FA
:060000000B308A00DB2B2F
:08000800F000030E8301F20079
:100010000A08F1008A0183130408F3000B1E182854
:100020008B1C18288B10831603179D17031383123C
:100030000C181B2828280C10831632087F39031D42
:10004000B203831283160130B007031856288301C8
:100050000B1F48288C1E482883161E303D020318AB
:1000600052283C08840083121A0880008316BC0AB8
:10007000DC303C02031C3E28BE30BC00BD0A0F3001
:100080003D02031C482803171D1C482883018614C1
:1000900083017308840071088A00720E8300F00ED9
:1000A000700E090083121A0883124828831704303F
:1000B000B100A13084000008F0390319682810301D
:1000C00080020008F039031D682884038001840A37
:1000D00010308407B10B5B28831327280F39820760
:1000E00030343134323433343434353436343734D4
:1000F000383439344134423443344434453446345A
:1001000083160130AC070318AD078312080083176C
:1001100003308407013080078403031880078403B9
:1001200003188007840303188007831308008317CC
:10013000033084073C0880078403013003188007DC
:1001400084030318800784030318800702308407A0
:100150003B088007840301300318800784030318D9
:100160008007831308000130D4070318D30703184E
:10017000D2070318D107D1282830BC020130031C54
:10018000BB023C08D40701300318D3070318D20779
:100190000318D1073B08D30701300318D20703180F
:1001A000D107780884000C30840783175108800039
:1001B000840A52088000840A53088000840A540884
:1001C000800083130800A701A801A901080083018A
:1001D0008701213060270C308A000230A000F02413
:1001E0008A010A308700000160270B308700000178
:1001F00060276B260C308700043060270D308700A5
:100200000001602725298701223060270C308700F4
:10021000043060270D308700000160270C308A0011
:100220006430A000F0248A01A03084000008840A11
:100230000004840A0004840A0004031D25298301A4
:1002400010308A00762001308A00831600303D028B
:10025000031D3B298030320203191F2983128A01B2
:10026000073087006D277C1AE728FC19E7287C19DE
:10027000E7283F292529831211308A004E2987015A
:1002800062306027073087006D277C08B100870146
:1002900022306027033087006D27FC0A80307C0203
:1002A000031C54294630FC0031087C02031925291F
:1002B000AD017C08AE001230AF00B0011127123042
:1002C000A6008313DE308400103087000910871EDB
:1002D0006729080809148000840AA60B662983167A
:1002E0005E1C7E2908306E02031D7E2900306F02DD
:1002F00003190A2A06306F0203199B29831303137B
:10030000831646305F02031CE72880305F02031823
:10031000E728DF0346305F02031890297F30DF00B3
:10032000831287012230602703308700DF3084008A
:10033000000860273A2983121230AD00E0308400B3
:100340000008AF00840A0008B0001230AF0201308C
:10035000031CB0021127393084002F083004031920
:10036000CB290910871EB229080809148000840AC5
:100370000130AF02031CB002841FAD292F083004E6
:100380000319CB290910871EC32909140130AF02B4
:10039000031CB002BE2900303F02031D7E2901303C
:1003A00040020319DB29023040020319D8297E29B3
:1003B00009308A001C29A030840051080002031D66
:1003C0007E29840A52080002031D7E29840A5308EC
:1003D0000002031D7E29840A54080002031D7E29A1
:1003E000992708304B2706304B2710308A009D2074
:1003F0008A0187012230602704308700403060275F
:10040000053087003C3060270630870000016027F8
:1004100089277E2983121230AD00E0308400000865
:10042000AF00840A0008B0001230AF020130031C94
:10043000B0021127393084000910871E1D2A0808D0
:1004400009148000840A0130AF02031CB00239088D
:10045000A6000F30A6050310A60DA60DA603422286
:1004600045303902031D402A063042020319812B10
:10047000113042020319C32A0130420203197C2AB7
:100480003D247E290910871E432A0808091480008C
:10049000840A0130AF02031CB002A60B422A0800F6
:1004A0002F08300403197A2A0910871E552A0808D4
:1004B00009148000840A0130AF02031CB00290309E
:1004C0000407031C502A2030840083172F083004AF
:1004D00003197A2A0910871E6B2A0808091480005C
:1004E000840A0130AF02031CB00290300407031CE1
:1004F000662A3D2483130800502208304D02031D54
:100500007E2900304E02031D7E290130B700AE2740
:100510002230AD004030AE003C08AF001330AF02D7
:10052000B001FB26E320103087003B273B273C0827
:10053000A6001830A602513084000008840A4B2718
:10054000903004070318BF2AA60B9D2A83130001CD
:100550004B272430AD004030AE00B8270430870070
:100560004030602705308700E030840000086027B5
:1005700006308700840A0008602789277E292030FA
:1005800084008317A42A0830A600422200304F02BC
:10059000031DE32A443050020319232BA0308400AA
:1005A00000084902031D7E29840A00084A02031D2F
:1005B0007E29840A00084B02031D7E29840A000854
:1005C0004C02031D7E29B530840000084F02031D34
:1005D000EE2A840A000850020319052BB730840064
:1005E00000084F02031DF92A840A0008500203196B
:1005F000082BB930840000084F02031D042B840A25
:100600000008500203190E2B7E2911308A00F729A9
:1006100055308400502208308A00202808308A0093
:10062000FC282F0830040319212B0910871E162BD4
:1006300008080914FC000130AF02031CB0020310CB
:100640000800031408005022A03084000008840A27
:100650000004840A0004840A0004031D7E290A3071
:100660008A004A2203308A0035304B2701304B275D
:1006700003304B273D304B2707304B2701304B27AA
:10068000A43084000630772736304B2704304B27C0
:10069000C0304B27A8304B2700304B2703304B2767
:1006A00032304B2704304B276530840004307727E5
:1006B000FF304B272330A60000014B27A60B5C2BF5
:1006C0000A308A00AD2203308A00A0308400650819
:1006D0008000840A66088000840A67088000840A13
:1006E000680880008316B20183120611C030A20090
:1006F0000C308A00DC240F308A00D42786018A015E
:100700007E291430A6004222B330840000084F0234
:10071000031D8F2B840A000850020319902B7E2999
:10072000A03084000008840A0004840A0004840ABB
:10073000000403197E29DA1A7E2909308A009A21D9
:1007400003308A000318A62BD6257E290C30840797
:1007500000085102031DBE2B840A00085202031D2B
:10076000BE2B840A00085302031DBE2B840A000816
:100770005402031DBE2B0F308402C0238A017E2940
:1007800003308A0000087F398207CE2BED2B022C24
:100790007E29DB2BE32B7E297E297E295A19D82B33
:1007A0005A18FC2B5A1E0800813080008313080061
:1007B0008001831308005A19D82B5A1E080085306F
:1007C0008000831308005A19D82B5A1C0800800196
:1007D0008313B3204F24080000005A19D82B5A184D
:1007E000FC2B840A03308A0000080F398207122C80
:1007F0002E2C332C382C072C003080008313B32090
:100800004F2408000030800083134C240800840328
:100810008430800083134C247808840008308407D7
:1008200087200800800A83130B308A0000230430DD
:100830008A0000307C020319262C0A307C0203193E
:10084000262C3F307C0203192B2C142C3D24BC2079
:100850001430FD008B2C0B308A00152B800A83137B
:100860001730FD008B2C800A83131A30FD008B2C6F
:10087000800A83131D30FD008B2C870122306027F6
:100880000A308700000160270B30870000016027D5
:1008900008000430B800512C1130B800512C103031
:1008A000B8000030BB002830BC000630B700AE27CF
:1008B0002230AD004030AE001430AF000030B00048
:1008C000FB26E320B3308400023077274D308400CC
:1008D00002307727780884000830840783170830AF
:1008E0007727831350304B2738084B2708304B2786
:1008F00000304B273B273B274726043087004030FA
:100900006027053087003C306027063087000001F3
:100910006027892708003F30FA000730FB002230AB
:10092000AD004030AE00FF30AF00FF30B000FB261E
:10093000AF01B001E320B3308400023080274D3096
:1009400084000230802783177808840008308407E9
:1009500004308027831351308400043080275030C6
:100960004527183045270830452700304527000126
:100970004527000145270001452700014527F901CA
:10098000031783127D088F000317831279088D00E7
:1009900083168C170C140000000083120E08F5005B
:1009A0000C08F6000313760DF50D7508FC007F307A
:1009B000FC05FC080319F82C24307C020319C72D10
:1009C00040307C020319892D25307C0203196D2DDE
:1009D0007E307C020319652D7C08452776087F3917
:1009E00045270130F9070317831203188F0AC42C17
:1009F0003D242F08BC003008BB0047261430BC073C
:100A000001300318BB070630B700AE27043087005B
:100A1000403060270E30BC0701300318BB0706309A
:100A200087003B086027BB080319262D0530870087
:100A30003C08602789273630BC020130031CBB020A
:100A40007808840008308407972008003C303C0276
:100A50000318162D053087003C30602789271B2D91
:100A6000F60DF60DF60D3830F6058130F6047608F1
:100A70009F000130A0000C308A00F02405308A006D
:100A80001F151F19412D1E08B30083161E0883125F
:100A9000B200F61E5F2D0310B20DB30D0310B20DA0
:100AA000B30D1E08B30783161E088312B20703187E
:100AB000B30A2030840083170D308A0074250D306E
:100AC0008A00142505308A00CF2D7F30F605F60EFA
:100AD0007608840083178313CF2D7F30F6057608C0
:100AE0008400840E0F3084058530840776087D25C8
:100AF0000008FC050319B22DB42DFD000130FC00E7
:100B00000730FD050319882D0310FC0DFD0B842D06
:100B100008007F30F60576088400840E0F308405C7
:100B2000031DA52D8530840776087D2500087C05EA
:100B30000319A42D1F308A001827FD0005308A00F4
:100B40007D08FC05031D302D8401053084077608DF
:100B50007D250008FC050319B82DB62D1F308A002D
:100B60007D0882003F30BA2D3B30BA2D3430BA2D8B
:100B70002D30BA2DFD00AE25FC0005308A00003076
:100B80007C020319CF2D7C084527FD0ABB2D0F30B1
:100B90008A0076087F39D03E122705308A0001305E
:100BA000F9070317831203188F0AC42CDA1C0800F4
:100BB00009308A00D12105308A000318492C003001
:100BC000BB002C30BC000630B700AE272230AD0091
:100BD0004030AE001830AF000030B000FB26E320FC
:100BE000B3308400023077274D30840002307727FD
:100BF000AA30840004307727B320780884000830B6
:100C00008407831783162A088000840A2B08800033
:100C1000840A2C088000840A2D088000840A83122C
:100C200051088000840A52088000840A530880001A
:100C3000840A5408800083137808840008308407ED
:100C40008720513084000430772760304B271230E2
:100C50004B2708304B2700304B273B273B270230E0
:100C60004B2704304B2705304B27B4304B27472602
:100C70000430870040306027053087003C30602713
:100C80000630870000016027892780200800A9011D
:100C9000A030840000082727840A00082727840A38
:100CA00000082727840A0008272745082727460821
:100CB0002727470827274808272700012727063026
:100CC0002727300827272F0827273230AD0040304C
:100CD000AE00B82708008726B426CB268316BE3080
:100CE000BC00BB00DC00BD01DD01831208008701F0
:100CF000213060271F3087006D271F3087007C0858
:100D00006027073087006D27FC1F812E080077269B
:100D10000E308700683060270A30870000016027A6
:100D20000B308700000160270130870046306027C4
:100D3000023087008030602703308700463060270C
:100D40000C308700003060270D30870002306027AC
:100D50000F3087001F30602707308700FF30602783
:100D60008701223060270800870122306027AD010B
:100D7000AE010C30AF00B00111270630A600A43040
:100D80008400103087006D276D277C088000840A5E
:100D9000A60BC12E08008701623060270130870052
:100DA000A43084000630A60000086027840A870A61
:100DB000A60BD42E07308700473060270830870005
:100DC00000016027870A00016027870A0001602769
:100DD000870A00016027870A00016027870A00014F
:100DE0006027870A00016027870A000160278701C2
:100DF000223060270800083087002D08602709305E
:100E000087002E0860270A3087002F0860270B30E4
:100E10008700300860278701123060271030870074
:100E20000800083087002D086027093087002E0849
:100E300060270A3087002F0860270B3087003008B2
:100E4000602787010A306027103087000800291CBE
:100E5000332FA70701300318A8070318A7070318A3
:100E6000A807A90A0800A80701300318A707031854
:100E7000A807A90A080000014B2700014B2F0130E9
:100E8000AF070318B00A7C084B2FFC000130AF07F6
:100E90000318B00A7C088800291C582FA7070130C6
:100EA0000318A8070318A7070318A807A90A612FA2
:100EB000A80701300318A7070318A807A90A612F7C
:100EC00088008316880183128910871E652F891474
:100ED0008316FF308800831208000910871E6E2FCA
:100EE0000808FC0009140800A03084000430A600A3
:100EF0001030870000084B27840AA60B7A2F0800C1
:100F0000A6001030870000084527840AA60B832F0F
:100F1000080087016D277C19892F870126306027FB
:100F2000043087006D277C18982FFC19892F902F8B
:100F300008002A30AF009E2F2230AF00B001AD0173
:100F40004030AE00FB2610308700E83084000630C9
:100F50007727A43084000630772708009C270830C4
:100F60004B2700304B27C5271830AD004030AE006E
:100F7000A709A8090230AF00B001FB261030870096
:100F800028086027270860270800E3201030870022
:100F900045304B2700304B273B084B273C084B275D
:100FA000AE30840000084B27840A00084B2701302C
:100FB000800784030318800700304B2700304B273D
:100FC000FF304B2737084B273B27742745308400D9
:060FD00004307727080041
:1010400008308A0055308400063000020318C52895
:101050000008840A82077F28312835284B286F280A
:1010600065283A207E0880047F283A20FE097E0801
:1010700080057F28840A0008FD000130FE00003052
:101080007D02031947280310FE0DFD033F2884034A
:101090000008840008000008AA00840A0008A600CE
:1010A000840A0008FD00840A0008FE00840A04087F
:1010B000FF002A08840000087D057E0480007F0868
:1010C0008400AA0AA60B51287F288316003000024C
:1010D000031D6C2881176D28811383127F28000857
:1010E0009F001F14840A0008A0000830A100A10B73
:1010F0007728A00B75281F151F197C288A01B73087
:10110000FF00BB012430BC008A011130B700AE27BC
:10111000E3202230AD004030AE001030AF00003090
:10112000B000FB26103087007F08840000084B27A2
:10113000840A00084B274D084B274E084B270030E8
:101140004B2710304B273B2705084B2706084B271A
:101150008530840000084B27840A00084B271E08AE
:10116000B30083161E088312B20033084B273208DF
:101170004B2783161F0883124B2700304B2708305C
:101180008A00C82008308A00ED2001308A007E29BC
:101190008A01A901A030840000082727840A0008DA
:1011A0002727840A00082727840A000827274508DC
:1011B0002727460827274708272748082727000109
:1011C000272711302727300827272F0827272830DF
:1011D000AD004030AE00B82708008A010430870017
:1011E00040306027053087003C306027063087009C
:1011F00000306027892708008316031710309E00EF
:1012000083015108B0005208AF000830AF02031C40
:10121000B00303308A00112309308A000318C5285F
:101220007C08D50004307C020318C5287C0882079E
:1012300038298D2997297129831341308400831619
:10124000031700089000840A00089100840A00082F
:101250009200840A00089300840A00089400840A1B
:1012600000089500830118160B1701308A007E29AB
:10127000BB012C30BC008A011130B700AE27E3203F
:101280002230AD004030AE001830AF000030B0006A
:10129000FB2610308700B930840000084B27840AF1
:1012A00000084B274D084B274E084B2700304B2793
:1012B00018304B273B278A0155084B2783179E3050
:1012C000840000084B27903084000E30772783136A
:1012D00008308A00C82008308A00ED2001308A00DA
:1012E0007E29831603179E01830103308A00112390
:1012F00009308A0003188A29831603171D1C8329C5
:10130000830106188A2983010527831603179E0A7D
:101310008301752909308A0038290630A600563025
:10132000840002308A00422210308A0000281030E7
:101330008A00682883170430F700A030F800780886
:101340008400801FCA290230840745080002031D5B
:10135000CA29840A46080002031DCA29840A4708CC
:101360000002031DCA29840A48080002031DCA2975
:10137000840A4D080002031DCA29840A4E0800028F
:10138000031DCA29840A07308402F03080048403D4
:10139000031408001030F807F70B9F29831303107C
:1013A00008008317A03084000408F8000430F70018
:1013B000801B0D2A80308000840AF0308000840A6F
:1013C00045088000840A46088000840A4708800097
:1013D000840A48088000840A4D088000840A4E0868
:1013E0008000840A51088000840A52088000840A20
:1013F00053088000840A54088000840A550880003D
:10140000840A56088000840A57088000840A580815
:101410008000840A83130310080010308407103002
:10142000F807F70BD8298313031408008A0100304A
:10143000AD004030AE002230AF000030B000FB26DF
:1014400010308700FF304B27FF304B27FF304B27F2
:10145000FF304B27FF304B27FF304B27A430840051
:1014600006307727080016228A0108304B27003003
:101470004B27FF30C500C600C700C8000130BB00C5
:101480004830BC001130B700C5271830AD004030DF
:10149000AE00B82F33228A01E3202230AD00403065
:1014A000AE003430AF000130B000FB2610308700B2
:1014B00000304B2744304B2700304B2743304B271D
:1014C00001304B2734304B273B2701304B2701306D
:1014D0004B2706304B2700014B27A630840000081D
:1014E0004B27840A00084B27840A00084B27840AEC
:1014F00000084B273B273B271030A60007308A0007
:1015000000014B270A308A00A60B7E2AA4308400F3
:1015100007308A00063077270A308A000A30A60092
:1015200007308A0000014B270A308A00A60B902A58
:10153000C030A60007308A0000014B270A308A001D
:10154000A60B9A2A07308A0063304B2782304B273C
:1015500053304B2763304B2708008A0100012727AF
:10156000000127270001272700012727FF30272711
:10157000FF302727FF302727FF30272700012727A5
:101580001130272701302727343027272830AD0096
:101590004030AE00B8270430870040306027053067
:1015A0008700563060270630870001306027892782
:1015B0000800D92A6230F9007F08FE067E08FF067F
:1015C0007F08FE06E5227F08FE00773079020319C6
:1015D000DA2A031783127D088D007E088C0083169B
:1015E0008C130C158B1355308D00AA308D008C1484
:1015F0008C18F82A0C1183120313FD0A8B170800AC
:101600002F0830040319132B0910871E052B080817
:101610000914FC000A307C020319132B0130AF02BD
:10162000031CB0020800FC010800002300307C020B
:101630000319792B0A307C020319792B49307C027B
:101640000319972B52307C020319A62B3030FC0271
:101650007C08FD00FD0E002300307C020319792B6D
:101660003030FC027C08FD04002300307C020319AA
:10167000792B7C08F900623079020319442B77300A
:1016800079020319442B792BFE01FF01002300305E
:101690007C020319792B26307C020319152B0023B9
:1016A00000307C020319792B20307C020319782B3F
:1016B00009307C020319782B26307C020319722B27
:1016C0002E307C020319742B2C307C020319742BEE
:1016D00030307C02031C742BC6307C070318742B3B
:1016E0007C234F2BE522152BE522FE01FF014F2B1A
:1016F000E52204308A00262C3030FC020310FE0D57
:10170000FF0D7E08F5007F08F6000310FE0DFF0DAB
:101710000310FE0DFF0D7508FE070318FF0A76087B
:10172000FF077C08FE070318FF0A0800962B992381
:10173000792B1830A600FD01D723FE000A308A005D
:10174000E9220B308A00A60B9C2B080000234130B5
:101750007C02031C792BBD307C070318792B4130A8
:10176000FC020530FC077C088400002330307C023A
:10177000031C792BC6307C070318792B3030FC0210
:10178000FC0AFD010314FD0DFC0BC32B00233D30AF
:101790007C02031D792B002348307C020319D42BD3
:1017A000FD097D088005792B7D088004792B1F3089
:1017B0008A007D0882008501860187018801073043
:1017C000890083168630620082309F003F3085009A
:1017D000003089008312A5016D2487248316350803
:1017E00036040F30031D033086008312031D2514B9
:1017F0009B24A224033089000530A000F024831626
:10180000E0308700FF3088000030890083125A24BE
:101810008A016B260C308A00A03084000008840AFC
:101820000004840A0004840A000403191B2C0F30EE
:101830008A00D4272C2C0C308A0006154430A200D4
:10184000DC244830A200DC244330A200DC245030E9
:10185000A200DC240C308A008316F030870083124B
:101860000C308A006430A000FE240C308A00071E71
:10187000A42D8316A030870026309800813099006F
:101880008C1683128030980083120B138A013F302C
:10189000FA000730FB008316B201831286018E0125
:1018A0008F010530900083160C1483120B178B17D1
:1018B0008B1703298317A03084004030F700800184
:1018C000840AF70B5F2C903084000E30F700800103
:1018D000840AF70B672C831308008316A03084005A
:1018E0000430FF00031783128D01031783168C1336
:1018F0000C1483120C088D0A03138000840AFF0B5A
:10190000752CAE3084008001840A80010800B33059
:1019100084000830FF000317831210308D008316F7
:101920008C130C1483120C088000840A8D0AFF0BA0
:101930008F2C031308008316AA01AB01AC01AD0183
:10194000831208000F30A000F02406113030A300ED
:10195000C8240530A000F0243030A300C82464302F
:10196000A000FE243030A300C8242030A300C824E7
:101970002830A200DC240130A200DC240230A000C8
:10198000F0240630A200DC240E30A200DC24080083
:10199000251CD82C0608A4000F30A405F030A305A0
:1019A0002308A40424088600D52C8615D72C86117C
:1019B0002830A000FE2408002208A300C824220822
:1019C000A300A30EC82408000615240E8A016E2069
:1019D000A200DC2424088A016E20A200DC24080076
:1019E0000030A100F32CF42CF52CF62CF72CF82C5D
:1019F000F92CA10BF22CA00BF02C0800FF2CA00B53
:101A0000FE2C08000408F400203084008317892588
:101A10008925892589258925892589258925892556
:101A200089250930B7002C2D0408F40020308400EB
:101A30008317742574257425742574250430B70024
:101A40002C2DB2000408F400203084008317602598
:101A5000602560250230B700B60100303602031D54
:101A6000352D3030000203193B2D0008FC005927AA
:101A70000D308A00B60A840AB70B2D2D0008FC0031
:101A800059270D308A008313740884000800B200BF
:101A90000408F40020308400831760256025602549
:101AA00006150008A200DC24840A0008A200DC2439
:101AB000840A0008A200DC24831374088400080050
:101AC0000830A600B6010310B20DB60DF630360789
:101AD0000318B6000318B20AA60B632D8403360858
:101AE00080003030800708001030A600B6010310D7
:101AF000B20DB30DB60DF63036070318B600031855
:101B0000B20AA60B772D8403360880003030800798
:101B100008002030A600B6010310B20DB30DB40DBD
:101B2000B50DB60DF63036070318B6000318B20A25
:101B3000A60B8C2D84033608800030308007080007
:101B400013308A007D0882000D308A00C030A20068
:101B50000611DC241030A6000030FD00A025A200F4
:101B60000D308A000615DC240D308A00FD0AA60B14
:101B7000AE2D8316A0308700263098008130990062
:101B80008C168312903098000530FA000F30FB005D
:101B90000B178B171030F700DF263330F700DF26E6
:101BA0002F30F700DF26831600303D020319D42DB5
:101BB0003B0884000008FC00BB0ADC303B02031C2D
:101BC000E32DBE30BB00BD0308307C020319F12DAC
:101BD0008312052783160D307C020319172EDD0AA8
:101BE000D42D00305D020319D42D3B0884008403FA
:101BF000BE3004020318FE2DDB30840080015C0837
:101C000084005D0884078403DC300402031C0A2E70
:101C1000BE30840280018313831205272030FC002C
:101C200005270830FC0005278316DD03D42D0A3074
:101C3000FC0083120527831600305D02031D362E3B
:101C400083122F30F700DF2683163B08DC00DD010E
:101C5000D42D83129230F700DF26202E1F308A0009
:101C60005E08432F1F308A005F0882005C08E00096
:101C70005D08E100DE012E26DF000E308A00003014
:101C80005F020319292E3226FD000E308A00003033
:101C90007D0203195E2EC82683160D307C020319BF
:101CA000572E7C087D02031D572EDF0A432E02307B
:101CB000DE076008DC006108DD003B2EDE0A2E2610
:101CC000FD0083120E308A007D0882009923333094
:101CD000F700DF26202E9C30F700DF26202EC826B6
:101CE00020307C0203196F2E09307C0203196F2EFD
:101CF00008001230FD00842E1430FD00842E1630B2
:101D0000FD00842E1030FD007730F9000130F8001E
:101D1000952E0430FD00912E0830FD00912E0030EC
:101D2000FD006230F9000430F8006F260D307C02AF
:101D30000319DB2E3D307C02031DDB2E6F260D3098
:101D40007C020319DB2EFE01FF01A72EC8260D30F1
:101D50007C020319C62E2E307C020319BD2E2C30B6
:101D60007C020319BD2E30307C02031CBD2EC63010
:101D70007C070318BD2E7C23A62EE522F803003035
:101D800078020319202EFE01FF01A62EE522202E47
:101D900083165C0884000008FC00DC0ADC305C026E
:101DA000031CD42EBE30DC00DD0300307C0203199E
:101DB000C92E831208008A30F700DF26202E031771
:101DC000831213308F0077088D0083168C170C1444
:101DD0000000000083120E08F5000C08F600031343
:101DE000760DF50D75087F390319042FFC0024309A
:101DF0007C0203190A2F052776087F390319042F5F
:101E0000FC000527F70ADF2E08000C1E052F7C08B2
:101E1000990008000F308A0076087F39D03E1227DB
:101E2000F70ADF2E8207A02F472F4A2F4E2F2D2F84
:101E3000312F352F392F522F1F2F3D2F432FAE30EB
:101E400084000008B300840A0008B200840A00304D
:101E5000B400840A0030B500022D031710308D0045
:101E60003C2F031712308D003C2F031714308D00C8
:101E70003C2F031716308D007B2FA03084000430D8
:101E8000FF0075270800031718308D00552F031722
:101E90008D01552F031704308D00552F031708307F
:101EA0008D00552F03170C308D000430FF00622F7A
:101EB00008007B088A007A0882002E30FC0059272F
:101EC0000F308A00031783168C130C1483120C082E
:101ED000FC008D0A03137C082125FF0B5D2F0800F1
:101EE0002E30FC0059270F308A000008840A212573
:101EF000FF0B702F0800031783168C130C1483122A
:101F00000C088D0A0313B300031783168C130C14EB
:101F100083120C088D0A0313B200142508008A01ED
:101F2000240E6E20FC000F308A0059278A012408F5
:101F30006E20FC000F308A0059270F308A000800FD
:101F4000A43084000008A400840A8F272D30FC00F0
:101F500059270F308A000008A400840A8F272D30EB
:101F6000FC0059270F308A000008A400840A8F273C
:101F70002D30FC0059270F308A000008A400840A85
:101F80008F272D30FC0059270F308A000008A4004D
:101F9000840A8F272D30FC0059270F308A00000853
:101FA000A400840A8F2708000D308A00A030840026
:101FB0000008840A47252E30A200DC240008840A89
:101FC00047252E30A200DC240008840A47252E3045
:0C1FD000A200DC240008840A4725080059
:102000000E30FD00FE018317903084000008FE04AE
:10201000840AFD0B0628831300307E02031D652809
:1020200083179630840056088000840A5708800081
:10203000840A58088000840A59088000840A4D08E0
:102040008000840A4E088000840A5A0880008316A3
:10205000000899008312840A5B08800000300002A7
:10206000031D0B1683138A01AD014030AE002A30E8
:10207000AF00B001FB2610308700FF304B27FF3048
:102080004B27FF304B27FF304B27FF304B27FF30CC
:102090004B27A43084000630772708304B270630C2
:1020A0004B2710308A00B8208A0187012230602730
:1020B0000430870040306027053087003C306027BF
:1020C0000630870000016027892709308A003829F7
:1020D00018120B130E30FD00FE01831790308400A0
:1020E0008001840AFD0B7028831365288316FF3056
:1020F000B20083120A308A004A228A0135304B2707
:1021000001304B2701304B273D304B2707304B2701
:1021100001304B27A430840006307727FF304B274F
:102120002F30A6008A0100014B2710308A00A60B31
:1021300092280A308A00AD2208008A0100014B274C
:1021400001304B2708304B2700304B2706304B27F8
:1021500004304B2700304B2702304B27A43084003B
:10216000063077277427413084000A30772708002B
:102170008A0100014B2701304B2708304B270030E4
:102180004B2706304B2704304B2700304B270130BC
:102190004B27A430840006307727742700304B2764
:1021A00000304B2700304B2700304B2700304B27A7
:1021B00000304B2783179630840010308A000317B5
:1021C000831204308D000313442183162008FE007F
:1021D0007D08FE050008FD05840A7E087D02031DBA
:1021E0002229442183162108FE007D08FE050008EF
:1021F000FD05840A7E087D02031D222944218316E1
:102200002208FE007D08FE050008FD05840A7E0800
:102210007D02031D2229442183162308FE007D0828
:10222000FE050008FD057E087D02031D222983129C
:1022300003138A019630840004307727831311300A
:102240008A0008000317831208308D0083160313D9
:1022500011308A0044218A017D084B2711308A0001
:1022600044218A017D084B2711308A0044218A01CC
:102270007D084B2711308A0044218A017D084B27B5
:10228000831311308A000800031783168C130C1473
:1022900083120C08FD008D0A031308008317903089
:1022A000840083160008E800840A0008E900840A14
:1022B0000008EA00840A0008EB00840A0008EC0029
:1022C000840A0008ED00840A83120008C500840A0D
:1022D0000008C600840A0008C700840A0008C80075
:1022E000840A831383163D08FD0083120030BB006F
:1022F0001C30BC007D08BC071030BC078A011130BF
:10230000B700AE27E3202230AD004030AE000830E9
:10231000AF001030AF077D08AF070030B000FB26DC
:1023200010308700B930840000084B27840A000869
:102330004B2783179A30840000084B27840A000833
:102340004B27831300304B2718307D074B273B2743
:1023500004304B277D08103E4B27831790308400B4
:102360000E307727831311308A0083163B088400D0
:102370000008FC00BB0ADC303B02031CC129BE3054
:10238000BB00BD0383128A017C084B2711308A00F1
:10239000FD0BB329861008308A00C8208A0104305A
:1023A0008700403060270E30BC0701300318BB07A0
:1023B000063087003B08602711308A00BB080319EC
:1023C000E9298A01053087003C08602789278A01AE
:1023D00025293C303C020318E1298A010530870099
:1023E0003C30602789278A0125298A017E295108E6
:1023F000B0005208AF000830AF02031CB003033036
:102400008A00112312308A000318F52901307C025A
:10241000031D282A03308A00112312308A00031872
:10242000F5290608FD0006117C08A2000C308A0080
:10243000DC2412308A007D088600FC30A205031DD2
:10244000282A0230A0000C308A00F02412308A00C2
:1024500003308A00112312308A0003183C2A060830
:10246000FD0006157C08A2000C308A00DC24123026
:102470008A007D088600282AB530FF0008308A00CF
:022480008128B1
:1026000042346F346F3474347334743472346134DC
:10261000703420344D346F346434653420342034C5
:102620008A068A064928A0216527773AF237A0351D
:10263000EE24653A6639E330A032E12164392D1089
:102640004210EF37733A723AF0304D10E437A0324F
:10265000652B7339EF34203738128A060000492879
:10266000CE21C324001F2A152A152015EF21663715
:10267000E734F23AF430EF3420372A152A152015C2
:102680008A06C126A021E420723220173A103012A7
:102690008A06C92DD02E411064322E393A103112DB
:1026A0008A06CE2DE52E4D3AF330A0353A1032127F
:1026B0008A06C72DE12E653AE12BA03C3A10331271
:1026C0008A06C82DF42E703A6F2874392010201015
:1026D000231034128A06CC2DC32E20226F28743981
:1026E00020102010231035128A06D02DE12E6139DA
:1026F0006C36EC326F287439231036128A06D32DCB
:10270000E52E6939EC306F28743920102310371208
:102710008A060000F9297437F83045107239F2370B
:102720000D170005EE24613B69362032EF21ED36AE
:10273000EE302E328A0600002A152A1520156F2148
:10274000F437F43961392038EF2665324810EC321D
:1027500020382A152A1520158A06EF316637E73406
:1027600020102010201020102D10501069397437BF
:102770004210E13764394310EE376933F53361397C
:10278000693AEE37611064375310613A753AAE39E1
:102790008A06F33D723ABD3EF63DEC30E53AA03E86
:1027A0002D1055106438F430A032F929F439ED3287
:1027B0004310EE376933F5336139693AEE37201744
:1027C0008A06EE34F434E1346936653D2010201079
:1027D0002D1041106C367210E732F334653A7339BC
:1027E0007310F43249106937693AEC305610EC3006
:0827F000E53AAE398A0600004B
:102800005424502AB1173017321030184F108D252C
:102810004305EE376537F431EF343A3763106F36DE
:10282000E5398A06EF217437EE322D3A793A653868
:10283000201D653A743CE8176D3A0D360D053C05D0
:102840005424CC263C1F4524C4203C1F492A4C2A32
:10285000BE224928A0216527773AF237A035EE2419
:10286000653A6639E330A032E12164392F1E492AE6
:102870004C2ABE222F1E4524C4203C1F4F21592222
:102880000A1F461ECE27202AC929452DAB1E3E19F8
:102890004928A0216527773AF237A035EE24653A1A
:1028A0006639E330A032E12164395610F232E93959
:1028B000EE37201038123C10C617CE273E2A481E8D
:1028C0003E29681EBE19AF24A0276F287439BC3971
:1028D000E817BE19441E3E26441E3E22461ED2273D
:1028E000A026C320492ACE27A21EEF3669327933AB
:1028F0006317E9332011C526482AC427A21EC52321
:10290000222A0A1F541EC22045264210D2274522E1
:102910003E29541E3E29541E3E226F2874392F1E14
:10292000442A3C1F442A561FEC30E53A2F1E442A05
:102930003C1FD4173E29541E3E29541E3E224129D5
:10294000201880123C10D4173E22541E2022CC2086
:10295000C7243D277211E73474343E1100202F1E26
:10296000442A3C1FD4173E29541E3E29541E3E22A1
:102970004129A01881123C10D4173E22541E202257
:10298000CC20C7243D277211E73474343E11012056
:102990002F1E442A3C1FD4173E29541E3E29541E84
:1029A0003E224129201982123C10D4173E22541E87
:1029B0002022CC20C7243D277211E73474343E1105
:1029C00002202F1E442A3C1FD4173E29541E3E29A4
:1029D000541E3E224129A01983123C10D4173E22D6
:1029E000541E2022CC20C7243D277211E7347434B2
:1029F0003E1103202F1E442A3C1FD4173E29541E8B
:102A00003E29541E3E224129A01A84123C10D4179C
:102A10003E22541E2022CC20C7243D277211E734C9
:102A200074343E1104204310EC32E939F33A2F1E7E
:0A2A3000442A3C1FD4173E29000081
:102E0000541E3E29541E3E224229201890123C1086
:102E1000D4173E22541E3E22491E5027D42A541055
:102E2000D02CBD227311E23AE936223A4E10CD2061
:102E3000BD22521130212011412B5526BD224811AF
:102E40003E111020491E5027D42A5410D02CBD22E8
:102E50007311E23AE936223A4E10CD20BD225211CA
:102E600030212011412B5526BD224C113E112F1E21
:102E7000442A3C1FD4173E29541E3E29541E3E228C
:102E80004229A01891123C10D4173E22541E3E2213
:102E9000491E5027D42A5410D02CBD227311E23A77
:102EA000E936223A4E10CD20BD2252113121201197
:102EB000412B5526BD2248113E111120491E502795
:102EC000D42A5410D02CBD227311E23AE936223AAA
:102ED0004E10CD20BD22521131212011412B5526FB
:102EE000BD224C113E112F1E442A3C1FD4173E29EF
:102EF000541E3E29541E3E224229201992123C1093
:102F0000D4173E22541E3E22491E5027D42A541064
:102F1000D02CBD227311E23AE936223A4E10CD2070
:102F2000BD22521132212011412B5526BD224811BC
:102F30003E111220491E5027D42A5410D02CBD22F5
:102F40007311E23AE936223A4E10CD20BD225211D9
:102F500032212011412B5526BD224C113E112F1E2E
:102F6000442A3C1FD4173E29541E3E29541E3E229B
:102F70004229A01993123C10D4173E22541E3E221F
:102F8000491E5027D42A5410D02CBD227311E23A86
:102F9000E936223A4E10CD20BD22521133212011A4
:102FA000412B5526BD2248113E111320491E5027A2
:102FB000D42A5410D02CBD227311E23AE936223AB9
:102FC0004E10CD20BD22521133212011412B552608
:102FD000BD224C113E112F1E442A3C1FD4173E29FE
:102FE000541E3E29541E3E224229201A94123C109F
:102FF000D4173E22541E3E22491E5027D42A541074
:10300000D02CBD227311E23AE936223A4E10CD207F
:10301000BD22521134212011412B5526BD224811C9
:103020003E111420491E5027D42A5410D02CBD2202
:103030007311E23AE936223A4E10CD20BD225211E8
:1030400034212011412B5526BD224C113E112F1E3B
:10305000442A3C1FD4173E29541E3E29541E3E22AA
:103060004229A01A95123C10D4173E22541E3E222B
:10307000491E5027D42A5410D02CBD227311E23A95
:10308000E936223A4E10CD20BD22521135212011B1
:10309000412B5526BD2248113E111520491E5027AF
:1030A000D42A5410D02CBD227311E23AE936223AC8
:1030B0004E10CD20BD22521135212011412B552615
:1030C000BD224C113E112F1E442A3C1FD4173E290D
:1030D000541E3E29541E3E224229201B96123C10AB
:1030E000D4173E22541E3E22491E5027D42A541083
:1030F000D02CBD227311E23AE936223A4E10CD208F
:10310000BD22521136212011412B5526BD224811D6
:103110003E111620491E5027D42A5410D02CBD220F
:103120007311E23AE936223A4E10CD20BD225211F7
:1031300036212011412B5526BD224C113E112F1E48
:10314000442A3C1FD4173E29541E3E29541E3E22B9
:103150004229A01B97123C10D4173E22541E3E2237
:10316000491E5027D42A5410D02CBD227311E23AA4
:10317000E936223A4E10CD20BD22521137212011BE
:10318000412B5526BD2248113E111720491E5027BC
:10319000D42A5410D02CBD227311E23AE936223AD7
:1031A0004E10CD20BD22521137212011412B552622
:1031B000BD224C113E112F1E442A3C1FD4173E291C
:1031C000541E3E29541E3E223C10D4173E22541E4B
:1031D0003E22491E5027D42A5410D02CBD227311F0
:1031E000E23AE936223A5610CC20C52AA21E6529B9
:1031F0006F36E4303E112F1E442A3C1FD4173E295F
:103200002F1E412A4C21BE222F1E4F234D293C1F29
:06321000C4173E26000079
:10340000461ED227A026C526482AC427A21EC523A9
:10341000222A4110D421CF243D277311E23AE93604
:103420002E3AE731A2340A1F681EBE19EF21663713
:10343000E734F23AF430EF343C37E817BE19441E53
:103440003E26441E3E22541EC22045264210D2274C
:1034500045223E29541E3E29541E3E22C126A0214B
:10346000E4207232F332BC39D4173E22541E3E227D
:1034700030122F1E442A3C1FD4173E29541E3E29C9
:10348000541E3E22D024411064323C39D4173E22CF
:10349000541E3E22491E5027D42A5410D02CBD223F
:1034A0007411F832223A4E10CD20BD22301162182C
:1034B00020115610CC20C52AA21E31123E112F1EFB
:1034C000442A3C1FD4173E29541E3E29541E3E2236
:1034D00065274D3AF330BC35D4173E22541E3E22A8
:1034E000491E5027D42A5410D02CBD227411F83212
:1034F000223A4E10CD20BD223011621A20115610F2
:10350000CC20C52AA21E32123E112F1E442A3C1F77
:10351000D4173E29541E3E29541E3E22E123653A0B
:10352000E12BBC3CD4173E22541E3E22491E50279C
:10353000D42A5410D02CBD227411F832223A4E10E5
:10354000CD20BD223011621C20115610CC20C52A7E
:10355000A21E33123E112F1E442A3C1FD4173E29AF
:10356000541E3E29541E3E227434703A5010F237D5
:10357000203A432A3A28BC11D4173E22541E3E2238
:10358000491E5027D42A5410D02CBD227411F83271
:10359000223A4E10CD20BD2231117718201156103D
:1035A000CC20C52AA21E34123E112F1E442A3C1FD5
:1035B000D4173E29541E3E29541E3E224326202263
:1035C0005010F237203AC42A3A28BC11D4173E22B0
:1035D000541E3E22491E5027D42A5410D02CBD22FE
:1035E0007411F832223A4E10CD20BD2231117719D4
:1035F00020115610CC20C52AA21E35123E112F1EB6
:10360000442A3C1FD4173E29541E3E29541E3E22F4
:10361000612861396C36EC325010F237203AC42AF6
:103620003A28BC11D4173E22541E3E22491E502770
:10363000D42A5410D02CBD227411F832223A4E10E4
:10364000CD20BD223111771A20115610CC20C52A69
:10365000A21E36123E112F1E442A3C1FD4173E29AB
:10366000541E3E29541E3E22E5296939EC30501083
:10367000F237203AC42A3A28BC11D4173E22541EED
:103680003E22491E5027D42A5410D02CBD2274113A
:10369000F832223A4E10CD20BD223111771B201175
:1036A0005610CC20C52AA21E37123E112F1E442AC6
:1036B0003C1FD4173E29541E3E29541E3E223C1066
:1036C000D4173E22541E3E22491E5027D42A54109D
:1036D000D02CBD227311E23AE936223A5610CC20A2
:1036E000C52AA21EE129653B3E11491E5027D42A56
:1036F0005410D02CBD227311E23AE936223A4E1012
:10370000CD20BD2249114927222A5610CC20C52A96
:10371000A21E65226133EC3A223A3E102F1E442A43
:103720003C1FD4173E292F1E412A4C21BE222F1E9A
:0C3730004F234D293C1FC4173E2600000B
:103A0000681EBE19F429F430F33A3C10E817BE19C9
:103A1000441E3E26441E3E22541EC220452642100D
:103A2000D22745223E29541E3E29541E3E22E52916
:103A300074375010E330E535733A3C10D4173E220A
:103A4000541E3E2239122F1E442A3C1FD4173E29F1
:103A5000541E3E29541E3E22682AF33449103C2845
:103A6000D4173E22541E3E223A122F1E442A3C1FD7
:103A7000D4173E292F1E412A4C21BE222F1E4C2234
:103A8000201F501E3C1F5224431FF037F23CE734E6
:103A900074342810A931321030182D18301931180B
:103AA0006210A03C411E481045293D236811743A1C
:103AB0003A38AF17F73BAE3B723AF334613A653AA6
:103AC0006E17AE3270353E11722AD334613A653AC0
:103AD0004310AE374C16643A3C17C117201F8A06B4
:103AE0002F1E4F2159223C1FC8174D2A3E26000089
:103E0000C034A8340034C834FF34FF34FF340034E5
:103E100000340034003400340134023400340034FF
:103E20000034503400340034273411342734123431
:103E300083161F0883120F398207FF34FF341F34A3
:103E40001F340B34033400340034F3343F3437343C
:103E50003334133403340134013420344C346F349C
:103E600077342034203400342034483469346734C3
:103E700068342034003449346E34203400344F34F4
:103E8000753474340034820778346634833466348D
:103E90006E3467347534673488346B348D346B34E6
:103EA0008F348F3492348F349434893498348934F5
:103EB0009A348C349F348C34A1348234A6348234C6
:103EC000A8347934AC347934AE347C34B7347C34AF
:103ED000B9347F34C0347F340034003463346F34F9
:103EE0006E3466346934673400346C3473340034AF
:103EF00069346E3469347434693461346C346934CF
:103F00007A346534003469346E346934743400347E
:103F1000683465346C34703400343F3400346934B0
:103F200070340034693400346E34653474340034D1
:103F30006E3400346734613474346534003467346B
:103F400000346834743474347034003468340034A9
:103F50006C346334643400346C3400347034613451
:103F6000723461346C346C3465346C3400347034C5
:103F70000034733465347234693461346C34003421
:043F80007334003462
:02400E00F23F7F
:10420000C000A8000000C800FF00FF00FF00000081
:10421000000000000000000001000200000000009B
:1042200000005000000000002700110027001200CD
:00000001FF
